:1000000000308A003E28000008308C00831605145A
:1000100083120518092890018C171C288C131C28A2
:10002000031005180314900C0C171C280C138C0BD0
:10003000102810088D0028281C308C1B07308D00DC
:100040008D0B202800008C1B0E280C1B1628102856
:10005000462810308400000803193D2801308D0027
:100060008C018C0B31288D0B30284A308C008C0B86
:10007000372800000000800B2E28512884011F30F3
:100080008305831685108312851404280D088F00BC
:1000900000308316860083120F08860064309000BB
:0600A00029284528630039
:00000001FF
